:020000040000FA
:0A000000000000007FEF01F08DD139
:08001800DAD1800E221A2150FA
:100020001D5C266E11E2266C1D5021C01DF0216E54
:100030001E5022C01EF0226E1F5023C01FF0236EE0
:10004000205024C020F0246E1A0E266074D0215255
:1000500072E0256A1E50286E2218296E1E8E228E8E
:10006000080E265E08E324C025F023C024F022C039
:1000700023F0226AF5D7262607E0D89022322332D1
:1000800024322532262EF9D729AE33D02450205ED3
:1000900023501F5A22501E5A07E2D880000E2056C5
:1000A0001F561E56800E281A256C04E02006000EEE
:1000B0001F5A1E5A040E266E1E660DD01FC01EF05B
:1000C00020C01FF025C020F0256A080E1D5E29E320
:1000D000262EF2D726D01EBE08D0D8902536203640
:1000E0001F361E361D2EF7D71CD025AE22D0256A0E
:1000F0000FD02450202623501F2222501E2206E318
:100100001E321F32203225321D4A0DD025AE11D0AD
:10011000203E0FD01F3E0DD01E3E0BD0D880209029
:10012000EFD71D6A02D027821D68206A1F6A800EE1
:100130001E6E28AE1E9E205012001E501C6E2218ED
:10014000296E1D50D8A421503AE01D267E0E03E3EF
:100150001D5E03E336D01D5E31E320C01AF01FC0E0
:100160001BF01C8E228E206A1F6A1E6A180E286ED3
:100170001C321B321A3206E32450202623501F2241
:1001800022501E221E321F322032282EF1D71EBED0
:1001900007D020361F361E361D5210E01D061C34B7
:1001A00016E3203E14D01F3E12D01E3E10D0D88041
:1001B0001E321F3220321D3E0AD003D027841D6A12
:1001C00002D027821D68206A1F6A800E1E6E29AE2B
:1001D0001E9E205012001DC028F01E5020C01EF090
:1001E000206E203628322032276A2036283602E355
:1001F0002784277E06E12780286A206A1F6A1E6AF4
:100200000BD0282803E0D880203206D0D8902032A6
:1002100002E1278201D0278627B604D027A20FD07B
:1002200027B407D07F0E206EFF0E1F6E1E6E1D6E50
:1002300023D0800E206E01D0206A000EF6D727B0A2
:10024000FBD71D6A9F0E2860EBD77E0E2864F4D77B
:100250009E0E285C07E0D89020321F321E321D32DD
:10026000282AF6D727A408D0D880000E1D561E567F
:100270001F56205620AEE0D71D5012001D6E1E6A7C
:100280001F6A206A299E0AD0299E20AE07D0D880F6
:10029000000E1D561E561F562056298E960E286E8D
:1002A000205209E0080E28261EC01DF01FC01EF0B7
:1002B00020C01FF011D01F520FE1080E285E1E5003
:1002C00007E1080E285E1D5002E1205010D01D6A83
:1002D0001F6E1DC01EF01D6A1FBE06D0D8901D36B1
:1002E0001E361F362806F8D729AE1F9E28501DC07F
:1002F00020F01D6E1F501EC01FF01E6E1200400E1B
:10030000276E4F0EAF6E240EAC6E900EAB6E0001DA
:10031000C69AC00E926E936A946E0F0EC16E070E4F
:10032000B46E6CD0F2A403D0F294827011009EAA35
:1003300019D0060EAB1412E1E2CF2BF0E1CF2AF078
:100340002C2A11EE00F02C50E126000EE222AECF56
:10035000E7FF2BC0E2FF2AC0E1FF1100AE50AE5014
:10036000AB98AB8811002C502D5C14E02D2AEACFFD
:100370000BF0E9CF0AF001EE00F02D50E926000E57
:10038000EA22EF500A6E0BC0EAFF0AC0E9FFD880EC
:10039000120004D0E8680A6ED8A0120012002C6A7D
:1003A0002D6A9D8A9F8AF28EF28C12009D9A01EE30
:1003B00000F0010EF46EF36AF306000EF45AEE6AD2
:1003C000F450F310F9E12C6A2D6A9D8A1200F29E16
:1003D000E0CFB4F4D8CFB5F4E8CFB6F4F28E000194
:1003E000A192F29EB4C4E0FFB5C4D8FFB6C4E8FF42
:1003F000F28E10009EA8FED7AD6E120092908990EA
:100400009296899693968A969292899292948994DA
:10041000939E8A9E92988998939C8A9C93988A9896
:1004200093948A94929A899A939A8A9A93928A92A6
:1004300093908A90949A8B9A94988B9894928B929A
:1004400094948B945A6A596A5C6A5B6A5E6A5D6AC4
:10045000606A5F6A626A616A646A636A666A656A38
:10046000686A676A6A6A696A6C6A6B6A6E6A6D6AE8
:10047000706A6F6A786A796A7A6A7B6A7C6A7D6A6E
:100480007E6A7F6A806B816B826B836B3A6A1FEC3A
:100490000EF01FEC10F0396A386A376A366A936AD0
:1004A0008A6A7DDF83DFCD6AF294F28A870ED56E89
:1004B000B16AA192B368E20EB26E00EE84F0300E23
:1004C000EE68E82EFDD77568748E3E6A3D6A3C6A18
:1004D0003B6A3F2AE86A3FB2010F40B0010806E1DB
:1004E00040703B2A000E3C223D223E223CDF2E6E15
:1004F000B60E2E5C06E3FE0E2E5CD8A0306A9CEF92
:1005000009F02EAE20D0306A850E2E5C04E12EC09C
:1005100030F0316814D0950E2E5C04E12EC030F01E
:1005200032680DD0A50E2E5C04E12EC030F0346888
:1005300006D0B50E2E5C03E12EC030F076689CEF3D
:1005400009F09AEF09F0305204E19CEF09F09AEFBC
:1005500009F0850E305CD8A4BFD0312805E12EC04B
:1005600031F09CEF09F0B6D0480E315C08E189907B
:10057000369038908769866985698469A8D0490E64
:10058000315C08E18996369238928B698A6989696B
:1005900088699DD04A0E315C08E18A963694389479
:1005A0008F698E698D698C6992D04B0E315C08E140
:1005B000899236963896936992699169906987D045
:1005C0004C0E315C08E136988994389897699669A1
:1005D000956994697CD04D0E315C08E1369A8A9E0B
:1005E000389A9B699A699969986971D04E0E315C05
:1005F00008E1369C8998389C9F699E699D699C6931
:1006000066D04F0E315C08E1369E8A9C389EA36905
:10061000A269A169A0695BD0500E315C08E13790F6
:100620008A983990A769A669A569A46950D0510E26
:10063000315C08E137928A943992AB69AA69A96959
:10064000A86945D0520E315C08E13794899A3994F3
:10065000AF69AE69AD69AC693AD0530E315C08E15F
:1006600037968A9A3996B369B269B169B0692FD061
:10067000540E315C03E0780E315C05E18A923168FA
:100680009CEF09F024D0550E315C03E0790E315C0B
:1006900005E18A9031689CEF09F019D0560E315C63
:1006A00003E07A0E315C05E18B9A31689CEF09F02A
:1006B0000ED0570E315C03E07B0E315C05E18B9868
:1006C00031689CEF09F003D031689CEF09F0316884
:1006D0009AEF09F09AEF09F0950E305CD8A46DEF0F
:1006E00008F0322804E12EC032F06CEF08F02EC082
:1006F00033F03352D8A4B6D0480E325C08E189906A
:10070000369038908769866985698469A8D0490ED2
:10071000325C08E18996369238928B698A698969D8
:1007200088699DD04A0E325C08E18A9636943894E6
:100730008F698E698D698C6992D04B0E325C08E1AD
:10074000899236963896936992699169906987D0B3
:100750004C0E325C08E1369889943898976996690E
:10076000956994697CD04D0E325C08E1369A8A9E78
:10077000389A9B699A699969986971D04E0E325C72
:1007800008E1369C8998389C9F699E699D699C699F
:1007900066D04F0E325C08E1369E8A9C389EA36973
:1007A000A269A169A0695BD0500E325C08E1379064
:1007B0008A983990A769A669A569A46950D0510E95
:1007C000325C08E137928A943992AB69AA69A969C7
:1007D000A86945D0520E325C08E13794899A399461
:1007E000AF69AE69AD69AC693AD0530E325C08E1CD
:1007F00037968A9A3996B369B269B169B0692FD0D0
:10080000540E325C03E0780E325C05E18A92326865
:100810009CEF09F024D0550E325C03E0790E325C77
:1008200005E18A9032689CEF09F019D0560E325CCF
:1008300003E07A0E325C05E18B9A32689CEF09F096
:100840000ED0570E325C03E07B0E325C05E18B98D4
:1008500032689CEF09F003D032689CEF09F03268EF
:100860009AEF09F032503A14016A006E0050480ABB
:100870000110D8A451D0898002EEB4F0D89033345E
:10088000E926000EEA22EECF41F0EFCF42F03680AB
:1008900041503B24046E42503C20056E000E3D202A
:1008A000066E000E3E20076E07C087F006C086F079
:1008B00005C085F004C084F078522CE0388003EE47
:1008C000B4F0D8907834E926000EEA22EECF04F096
:1008D000EFCF05F0D8904134086E4234096E0450D1
:1008E000085C0550095805E342C05AF041C059F070
:1008F00011D003EEB4F0D8907834E926000EEA2245
:10090000EECF04F0EFCF05F04150045C596E425039
:1009100005585A6E6AEF08F00050490A0110D8A431
:1009200051D0898602EEB4F0D8903334E926000E17
:10093000EA22EECF43F0EFCF44F0368243503B241F
:10094000046E44503C20056E000E3D20066E000EE5
:100950003E20076E07C08BF006C08AF005C089F004
:1009600004C088F079522CE0388203EEB4F0D890BD
:100970007934E926000EEA22EECF04F0EFCF05F03D
:10098000D8904334086E4434096E0450085C055016
:10099000095805E344C05CF043C05BF011D003EE9E
:1009A000B4F0D8907934E926000EEA22EECF04F0B4
:1009B000EFCF05F04350045C5B6E445005585C6E0D
:1009C0006AEF08F000504A0A0110D8A451D08A8674
:1009D00002EEB4F0D8903334E926000EEA22EECFCE
:1009E00045F0EFCF46F0368445503B24046E465028
:1009F0003C20056E000E3D20066E000E3E20076E68
:100A000007C08FF006C08EF005C08DF004C08CF0DA
:100A10007A522CE0388403EEB4F0D8907A34E92688
:100A2000000EEA22EECF04F0EFCF05F0D890453467
:100A3000086E4634096E0450085C0550095805E3F9
:100A400046C05EF045C05DF011D003EEB4F0D89022
:100A50007A34E926000EEA22EECF04F0EFCF05F05B
:100A60004550045C5D6E465005585E6E6AEF08F0B6
:100A700000504B0A0110D8A451D0898202EEB4F084
:100A8000D8903334E926000EEA22EECF47F0EFCFBC
:100A900048F0368647503B24046E48503C20056E93
:100AA000000E3D20066E000E3E20076E07C093F03C
:100AB00006C092F005C091F004C090F07B522CE08B
:100AC000388603EEB4F0D8907B34E926000EEA2293
:100AD000EECF04F0EFCF05F0D8904734086E4834DD
:100AE000096E0450085C0550095805E348C060F0E1
:100AF00047C05FF011D003EEB4F0D8907B34E92604
:100B0000000EEA22EECF04F0EFCF05F04750045C70
:100B10005F6E48500558606E6AEF08F000504C0A4E
:100B20000110D8A451D002EEB4F0D8903334E926A5
:100B3000000EEA22EECF49F0EFCF4AF089843688E2
:100B400049503B24046E4A503C20056E000E3D2067
:100B5000066E000E3E20076E07C097F006C096F0A6
:100B600005C095F004C094F07C522CE0388803EE68
:100B7000B4F0D8907C34E926000EEA22EECF04F0DF
:100B8000EFCF05F0D8904934086E4A34096E04500E
:100B9000085C0550095805E34AC062F049C061F09D
:100BA00011D003EEB4F0D8907C34E926000EEA228E
:100BB000EECF04F0EFCF05F04950045C616E4A506F
:100BC0000558626E6AEF08F000504D0A0110D8A473
:100BD00051D002EEB4F0D8903334E926000EEA2268
:100BE000EECF4BF0EFCF4CF08A8E368A4B503B2441
:100BF000046E4C503C20056E000E3D20066E000E2B
:100C00003E20076E07C09BF006C09AF005C099F021
:100C100004C098F07D522CE0388A03EEB4F0D890EE
:100C20007D34E926000EEA22EECF04F0EFCF05F086
:100C3000D8904B34086E4C34096E0450085C055053
:100C4000095805E34CC064F04BC063F011D003EECB
:100C5000B4F0D8907D34E926000EEA22EECF04F0FD
:100C6000EFCF05F04B50045C636E4C500558646E3A
:100C70006AEF08F000504E0A0110D8A450D002EEDE
:100C8000B4F0D8903334E926000EEA22EECF4DF0CE
:100C9000EFCF4EF08988368C4D503B24046E4E5079
:100CA0003C20056E000E3D20066E000E3E20076EB5
:100CB00007C09FF006C09EF005C09DF004C09CF0E8
:100CC0007E522CE0388C03EEB4F0D8907E34E926C6
:100CD000000EEA22EECF04F0EFCF05F0D8904D34AD
:100CE000086E4E34096E0450085C0550095805E33F
:100CF0004EC066F04DC065F011D003EEB4F0D89050
:100D00007E34E926000EEA22EECF04F0EFCF05F0A4
:100D10004D50045C656E4E500558666EDBD1005038
:100D20004F0A0110D8A450D002EEB4F0D89033345A
:100D3000E926000EEA22EECF4FF0EFCF50F08A8C7A
:100D4000368E4F503B24046E50503C20056E000EF2
:100D50003D20066E000E3E20076E07C0A3F006C0C1
:100D6000A2F005C0A1F004C0A0F07F522CE0388EA4
:100D700003EEB4F0D8907F34E926000EEA22EECFDD
:100D800004F0EFCF05F0D8904F34086E5034096E60
:100D90000450085C0550095805E350C068F04FC086
:100DA00067F011D003EEB4F0D8907F34E926000E3E
:100DB000EA22EECF04F0EFCF05F04F50045C676EEF
:100DC00050500558686E86D10050500A0110D8A4C2
:100DD00050D002EEB4F0D8903334E926000EEA2267
:100DE000EECF51F0EFCF52F08A88378051503B243C
:100DF000046E52503C20056E000E3D20066E000E23
:100E00003E20076E07C0A7F006C0A6F005C0A5F0FB
:100E100004C0A4F080532CE0398003EEB4F0D890E5
:100E20008035E926000EEA22EECF04F0EFCF05F080
:100E3000D8905134086E5234096E0450085C055045
:100E4000095805E352C06AF051C069F011D003EEB1
:100E5000B4F0D8908035E926000EEA22EECF04F0F7
:100E6000EFCF05F05150045C696E525005586A6E20
:100E700031D10050510A0110D8A450D002EEB4F084
:100E8000D8903334E926000EEA22EECF53F0EFCFAC
:100E900054F08A84378253503B24046E54503C20D3
:100EA000056E000E3D20066E000E3E20076E07C048
:100EB000ABF006C0AAF005C0A9F004C0A8F08153A9
:100EC0002CE0398203EEB4F0D8908135E926000E8B
:100ED000EA22EECF04F0EFCF05F0D8905334086E3D
:100EE0005434096E0450085C0550095805E354C099
:100EF0006CF053C06BF011D003EEB4F0D890813594
:100F0000E926000EEA22EECF04F0EFCF05F05350B1
:100F1000045C6B6E545005586C6EDCD00050520A65
:100F20000110D8A450D002EEB4F0D8903334E926A2
:100F3000000EEA22EECF55F0EFCF56F0898A3784C3
:100F400055503B24046E56503C20056E000E3D204B
:100F5000066E000E3E20076E07C0AFF006C0AEF072
:100F600005C0ADF004C0ACF082532CE0398403EE30
:100F7000B4F0D8908235E926000EEA22EECF04F0D4
:100F8000EFCF05F0D8905534086E5634096E0450F2
:100F9000085C0550095805E356C06EF055C06DF069
:100FA00011D003EEB4F0D8908235E926000EEA2283
:100FB000EECF04F0EFCF05F05550045C6D6E565047
:100FC00005586E6E87D00050530A0110D8A450D037
:100FD00002EEB4F0D8903334E926000EEA22EECFC8
:100FE00057F0EFCF58F08A8A378657503B24046E6B
:100FF00058503C20056E000E3D20066E000E3E202F
:10100000076E07C0B3F006C0B2F005C0B1F004C06F
:10101000B0F083532CE0398603EEB4F0D8908335DA
:10102000E926000EEA22EECF04F0EFCF05F0D890CB
:101030005734086E5834096E0450085C055009583E
:1010400005E358C070F057C06FF011D003EEB4F054
:10105000D8908335E926000EEA22EECF04F0EFCFD8
:1010600005F05750045C6F6E58500558706E32D0C2
:101070000050540A011004E00050780A011004E105
:101080008A82326859D126D00050550A011004E0F6
:101090000050790A011004E18A8032684DD11AD0DB
:1010A0000050560A011004E000507A0A011004E1D1
:1010B0008B8A326841D10ED00050570A011004E0EB
:1010C00000507B0A011004E18B88326835D102D0D0
:1010D000326832D132682ED12DD1A50E305CD8A421
:1010E0001CD1342804E12EC034F026D115D1480E8D
:1010F000345C14E12EC078F078520CE003EEB4F0CA
:10110000D8907834E926000EEA22EECF59F0EFCFDE
:101110005AF003D05A6A596A3890FCD0490E345CB0
:1011200014E12EC079F079520CE003EEB4F0D890BF
:101130007934E926000EEA22EECF5BF0EFCF5CF0C7
:1011400003D05C6A5B6A3892E5D04A0E345C14E1E5
:101150002EC07AF07A520CE003EEB4F0D8907A34D4
:10116000E926000EEA22EECF5DF0EFCF5EF003D06D
:101170005E6A5D6A3894CED04B0E345C14E12EC0AA
:101180007BF07B520CE003EEB4F0D8907B34E92680
:10119000000EEA22EECF5FF0EFCF60F003D0606A7E
:1011A0005F6A3896B7D04C0E345C14E12EC07CF0E8
:1011B0007C520CE003EEB4F0D8907C34E926000EAB
:1011C000EA22EECF61F0EFCF62F003D0626A616A8B
:1011D0003898A0D04D0E345C14E12EC07DF07D52C5
:1011E0000CE003EEB4F0D8907D34E926000EEA223C
:1011F000EECF63F0EFCF64F003D0646A636A389A8D
:1012000089D04E0E345C14E12EC07EF07E520CE08C
:1012100003EEB4F0D8907E34E926000EEA22EECF39
:1012200065F0EFCF66F003D0666A656A389C72D0CD
:101230004F0E345C14E12EC07FF07F520CE003EEC1
:10124000B4F0D8907F34E926000EEA22EECF67F0A2
:10125000EFCF68F003D0686A676A389E5BD0500EA3
:10126000345C14E12EC080F080530CE003EEB4F047
:10127000D8908035E926000EEA22EECF69F0EFCF54
:101280006AF003D06A6A696A399044D0510E345CBE
:1012900014E12EC081F081530CE003EEB4F0D8903D
:1012A0008135E926000EEA22EECF6BF0EFCF6CF02D
:1012B00003D06C6A6B6A39922DD0520E345C14E103
:1012C0002EC082F082530CE003EEB4F0D890823549
:1012D000E926000EEA22EECF6DF0EFCF6EF003D0DC
:1012E0006E6A6D6A399416D0530E345C13E12EC0C9
:1012F00083F083530CE003EEB4F0D8908335E926F5
:10130000000EEA22EECF6FF0EFCF70F003D0706ADC
:101310006F6A3996346810D00DD0B50E305C0AE192
:10132000762804E12EC076F007D004D02EC077F0E6
:10133000E3EC0CF0A9EC0CF00C0E755CD8B0A0EF4F
:101340000CF071503B5C72503C5873503D587450D7
:101350003E58D8A07FEF0CF0748E75523AE138B049
:1013600007D03690899087698669856984692FD00E
:1013700036A017D0899059503B24006E5A503C201B
:10138000016E000E3D20026E000E3E20036E03C073
:1013900087F002C086F001C085F000C084F036906E
:1013A00016D0898041503B24006E42503C20016E93
:1013B000000E3D20026E000E3E20036E03C087F03B
:1013C00002C086F001C085F000C084F036807EEF58
:1013D0000CF0010E755C3AE138B207D0369289966E
:1013E0008B698A69896988692FD036A217D0899656
:1013F0005B503B24006E5C503C20016E000E3D2093
:10140000026E000E3E20036E03C08BF002C08AF015
:1014100001C089F000C088F0369216D0898643500A
:101420003B24006E44503C20016E000E3D20026EB5
:10143000000E3E20036E03C08BF002C08AF001C094
:1014400089F000C088F036827EEF0CF0020E755CE9
:101450003AE138B407D036948A968F698E698D69DF
:101460008C692FD036A417D08A965D503B24006E2D
:101470005E503C20016E000E3D20026E000E3E20AC
:10148000036E03C08FF002C08EF001C08DF000C06B
:101490008CF0369416D08A8645503B24006E465018
:1014A0003C20016E000E3D20026E000E3E20036EB9
:1014B00003C08FF002C08EF001C08DF000C08CF030
:1014C00036847EEF0CF0030E755C39E138B607D038
:1014D0003696899293699269916990692FD036A660
:1014E00017D089925F503B24006E60503C20016E03
:1014F000000E3D20026E000E3E20036E03C093F0EE
:1015000002C092F001C091F000C090F0369616D063
:10151000898247503B24006E48503C20016E000EEB
:101520003D20026E000E3E20036E03C093F002C009
:1015300092F001C091F000C090F03686DFD1040E29
:10154000755C39E138B807D03698899497699669FF
:10155000956994692FD036A817D0899461503B249F
:10156000006E62503C20016E000E3D20026E000EA7
:101570003E20036E03C097F002C096F001C095F0C4
:1015800000C094F0369816D0898449503B24006EF0
:101590004A503C20016E000E3D20026E000E3E209F
:1015A000036E03C097F002C096F001C095F000C032
:1015B00094F03688A3D1050E755C39E138BA07D0AE
:1015C000369A8A9E9B699A69996998692FD036AA3A
:1015D00017D08A9E63503B24006E64503C20016EFD
:1015E000000E3D20026E000E3E20036E03C09BF0F5
:1015F00002C09AF001C099F000C098F0369A16D057
:101600008A8E4B503B24006E4C503C20016E000EE5
:101610003D20026E000E3E20036E03C09BF002C010
:101620009AF001C099F000C098F0368A67D1060E92
:10163000755C39E138BC07D0369C89989F699E69F2
:101640009D699C692FD036AC17D0899865503B2492
:10165000006E66503C20016E000E3D20026E000EB2
:101660003E20036E03C09FF002C09EF001C09DF0BB
:1016700000C09CF0369C16D089884D503B24006EEB
:101680004E503C20016E000E3D20026E000E3E20AA
:10169000036E03C09FF002C09EF001C09DF000C029
:1016A0009CF0368C2BD1070E755C39E138BE07D023
:1016B000369E8A9CA369A269A169A0692FD036AE23
:1016C00017D08A9C67503B24006E68503C20016E06
:1016D000000E3D20026E000E3E20036E03C0A3F0FC
:1016E00002C0A2F001C0A1F000C0A0F0369E16D04A
:1016F0008A8C4F503B24006E50503C20016E000EEF
:101700003D20026E000E3E20036E03C0A3F002C017
:10171000A2F001C0A1F000C0A0F0368EEFD0080EFC
:10172000755C39E139B007D037908A98A769A66906
:10173000A569A4692FD037A017D08A9869503B2497
:10174000006E6A503C20016E000E3D20026E000EBD
:101750003E20036E03C0A7F002C0A6F001C0A5F0B2
:1017600000C0A4F0379016D08A8851503B24006EF8
:1017700052503C20016E000E3D20026E000E3E20B5
:10178000036E03C0A7F002C0A6F001C0A5F000C020
:10179000A4F03780B3D0090E755C39E139B207D0B7
:1017A00037928A94AB69AA69A969A8692FD037A230
:1017B00017D08A946B503B24006E6C503C20016E15
:1017C000000E3D20026E000E3E20036E03C0ABF003
:1017D00002C0AAF001C0A9F000C0A8F0379216D04C
:1017E0008A8453503B24006E54503C20016E000EFE
:1017F0003D20026E000E3E20036E03C0ABF002C01F
:10180000AAF001C0A9F000C0A8F0378277D00A0E74
:10181000755C39E139B407D03794899AAF69AE69FC
:10182000AD69AC692FD037A417D0899A6D503B248D
:10183000006E6E503C20016E000E3D20026E000EC8
:101840003E20036E03C0AFF002C0AEF001C0ADF0A9
:1018500000C0ACF0379416D0898A55503B24006EF6
:1018600056503C20016E000E3D20026E000E3E20C0
:10187000036E03C0AFF002C0AEF001C0ADF000C017
:10188000ACF037843BD00B0E755C38E139B607D02D
:1018900037968A9AB369B269B169B0692FD037A611
:1018A00017D08A9A6F503B24006E70503C20016E16
:1018B000000E3D20026E000E3E20036E03C0B3F00A
:1018C00002C0B2F001C0B1F000C0B0F0379616D03F
:1018D0008A8A57503B24006E58503C20016E000EFF
:1018E0003D20026E000E3E20036E03C0B3F002C026
:1018F000B2F001C0B1F000C0B0F037862AD83EAED9
:101900001ED03E6A3D6A3C6A3B6A376A366A396A6B
:10191000386A00EE84F0300EEE68E82EFDD789902C
:1019200089968A96899289948A9E89988A9C8A98AF
:101930008A94899A8A9A8A928A908B9A8B9806D0EE
:101940003EAE04D03E6A3D6A3C6A3B6A827669EFED
:1019500002F07568748E2F6A0C0E2F5C33E2D890FB
:101960002F34E96EEA6AEA36E936EA36840EE92669
:10197000000EEA22EFCF00F0ECCF01F0ECCF02F046
:10198000ECCF03F07150005C725001587350025854
:101990007450035815E2D8902F34E96EEA6AEA369B
:1019A000E936EA36840EE926000EEA22EFCF71F01E
:1019B000ECCF72F0ECCF73F0ECCF74F02FC075F079
:1019C0002F2ACAE312001E0E765CD8A4C6D0775226
:1019D00027E1396A386A5A6A596A786A5C6A5B6AC6
:1019E000796A5E6A5D6A7A6A606A5F6A7B6A626A5D
:1019F000616A7C6A646A636A7D6A666A656A7E6A2D
:101A0000686A676A7F6A6A6A696A806B6C6A6B6A0D
:101A1000816B6E6A6D6A826B706A6F6A836B9CD031
:101A200077C078F003EEB4F0D8907734E926000E52
:101A3000EA22EECF59F0EFCF5AF077C079F003EEFB
:101A4000B4F0D8907734E926000EEA22EECF5BF0AE
:101A5000EFCF5CF077C07AF003EEB4F0D890773433
:101A6000E926000EEA22EECF5DF0EFCF5EF077C000
:101A70007BF003EEB4F0D8907734E926000EEA222A
:101A8000EECF5FF0EFCF60F077C07CF003EEB4F004
:101A9000D8907734E926000EEA22EECF61F0EFCF3E
:101AA00062F077C07DF003EEB4F0D8907734E92689
:101AB000000EEA22EECF63F0EFCF64F077C07EF045
:101AC00003EEB4F0D8907734E926000EEA22EECF88
:101AD00065F0EFCF66F077C07FF003EEB4F0D890FA
:101AE0007734E926000EEA22EECF67F0EFCF68F0F8
:101AF00077C080F003EEB4F0D8907734E926000E7A
:101B0000EA22EECF69F0EFCF6AF077C081F003EE02
:101B1000B4F0D8907734E926000EEA22EECF6BF0CD
:101B2000EFCF6CF077C082F003EEB4F0D89077344A
:101B3000E926000EEA22EECF6DF0EFCF6EF077C00F
:101B400083F003EEB4F0D8907734E926000EEA2251
:101B5000EECF6FF0EFCF70F070D0420E765CD8A46D
:101B60004AD07752D8A445D0376A366A396A386A7B
:101B700000EE84F0300EEE68E82EFDD7756889908F
:101B800089968A96899289948A9E89988A9C8A984D
:101B90008A94899A8A9A5A6A596A5C6A5B6A5E6A06
:101BA0005D6A606A5F6A626A616A646A636A666AD9
:101BB000656A686A676A6A6A696A6C6A6B6A6E6A89
:101BC0006D6A706A6F6A786A796A7A6A7B6A7C6A17
:101BD0007D6A7E6A7F6A806B816B826B836B3A6AF7
:101BE0003E6A3D6A3C6A3B6A8A928A908B9A8B98DD
:101BF00001D03A6822D07B0E765C1FE1376A366AE4
:101C0000396A386A899089968A96899289948A9ED7
:101C100089988A9C8A988A94899A8A9A3E6A3D6AA7
:101C20003C6A3B6A00EE84F0300EEE68E82EFDD789
:101C300075688A928A908B9A8B9876681200030155
:101C4000B569B469A20EB76FC30EB66F9A0EB96FBD
:101C5000460EB86F960EBB6F320EBA6F920EBD6F06
:101C60003A0EBC6F8E0EBF6F5D0EBE6F8A0EC16FD7
:101C70009A0EC06F860EC36FF00EC26F830EC56FD3
:101C80005F0EC46F7F0EC76FE70EC66F7C0EC96F05
:101C9000850EC86F790ECB6F3B0ECA6F760ECD6F77
:101CA000070ECC6F720ECF6FE80ECE6F6F0ED16F36
:101CB000DF0ED06F6C0ED36FEA0ED26F6A0ED56F47
:101CC0000A0ED46F670ED76F3C0ED66F640ED96FB5
:101CD000820ED86F610EDB6FDA0EDA6F5F0EDD6F8A
:101CE000440EDC6F5C0EDF6FBF0EDE6F5A0EE16FCD
:101CF0004C0EE06F570EE36FE90EE26F550EE56F85
:101D0000960EE46F530EE76FE66F510EE96F200EEB
:101D1000E86F4E0EEB6FFB0EEA6F4C0EED6FE50EAB
:101D2000EC6F4A0EEF6FDC0EEE6F480EF16FE20EB5
:101D3000F06F460EF36FF50EF26F450EF56F150E50
:101D4000F46F430EF76F420EF66F410EF96F7B0E84
:101D5000F86F3F0EFB6FC00EFA6F3E0EFD6F100E58
:101D6000FC6F3C0EFF6F6D0EFE6F3A0E0401016FAB
:101D7000D40E006F390E036F460E026F370E056FDB
:101D8000C20E046F360E076F490E066F340E096FD0
:101D9000DA0E086F330E0B6F740E0A6F320E0D6F72
:101DA000180E0C6F300E0F6FC50E0E6F2F0E116FC9
:101DB0007B0E106F2E0E136F3A0E126F2D0E156FD5
:101DC000020E146F2B0E176FD10E166F2A0E196F9D
:101DD000A90E186F290E1B6F880E1A6F280E1D6F23
:101DE0006F0E1C6F270E1F6F5E0E1E6F260E216F6B
:101DF000530E206F250E236F500E226F240E256F79
:101E0000540E246F230E276F5E0E266F220E296F4D
:101E10006F0E286F210E2B6F860E2A6F200E2D6FEE
:101E2000A30E2C6F1F0E2F6FC60E2E6F1E0E316F5E
:101E3000EF0E306F1E0E336F326F1D0E356F520E68
:101E4000346F1C0E376F8C0E366F1B0E396FCB0E36
:101E5000386F1B0E3B6F0F0E3A6F1A0E3D6F580E08
:101E60003C6F190E3F6FA50E3E6F180E416FF80EB6
:101E7000406F180E436F4F0E426F170E456FAB0E3B
:101E8000446F170E476F0A0E466F160E496F6F0E9E
:101E9000486F150E4B6FD70E4A6F150E4D6F430EE0
:101EA0004C6F140E4F6FB30E4E6F140E516F270E02
:101EB000506F130E536F9F0E526F130E556F1A0E05
:101EC000546F120E576F990E566F120E596F1B0EEC
:101ED000586F110E5B6FA10E5A6F110E5D6F290EB8
:101EE0005C6F100E5F6FB50E5E6F100E616F440E6B
:101EF000606F0F0E636FD60E626F0F0E656F6B0E05
:101F0000646F0F0E676F030E666F0E0E696F9D0E86
:101F1000686F0E0E6B6F3A0E6A6F0D0E6D6FDA0EF4
:101F20006C6F0D0E6F6F7C0E6E6F0D0E716F210E4C
:101F3000706F0C0E736FC80E726F0C0E756F720E91
:101F4000746F0C0E776F1E0E766F0B0E796FCC0EC2
:101F5000786F0B0E7B6F7C0E7A6F0B0E7D6F2E0EE3
:101F60007C6F0A0E7F6FE30E7E6F0A0E816F990EF3
:101F7000806F0A0E836F510E826F0A0E856F0B0EF3
:101F8000846F090E876FC80E866F090E896F850EE4
:101F9000886F090E8B6F450E8A6F090E8D6F060EC6
:101FA0008C6F080E8F6FC90E8E6F080E916F8E0E9C
:101FB000906F080E936F540E926F080E956F1C0E63
:101FC000946F070E976FE50E966F070E996FAF0E21
:101FD000986F070E9B6F7B0E9A6F070E9D6F490ED1
:101FE0009C6F070E9F6F170E9E6F060EA16FE70E78
:101FF000A06F060EA36FB90EA26F060EA56F8B0E13
:10200000A46F060EA76F5F0EA66F060EA96F340EA3
:10201000A86F060EAB6F0A0EAA6F050EAD6FE10E2C
:10202000AC6F050EAF6FB90EAE6F050EB16F930EAC
:10203000B06F050EB36F6D0EB26F00011200010E8E
:102040002F6E800E2F5CD8B06FD0116A106A180EF8
:102050000F6E850E0E6ECD0E156ECC0E146E0A0E22
:10206000136E830E126E2F503EEC01F020C019F05B
:102070001FC018F01EC017F01DC016F0246A236A96
:10208000226A7F0E216E19C020F018C01FF017C001
:102090001EF016C01DF00DEC00F020C019F01FC09E
:1020A00018F01EC017F01DC016F015C024F014C0A3
:1020B00023F013C022F012C021F019C020F018C084
:1020C0001FF017C01EF016C01DF09DEC00F020C0E0
:1020D00015F01FC014F01EC013F01DC012F011C087
:1020E00024F010C023F00FC022F00EC021F015C064
:1020F00020F014C01FF013C01EF012C01DF00FEC32
:1021000000F0EBEC00F0006E1EC001F002EEB4F047
:10211000D8902F34E926000EEA2200C0EEFF01C05D
:0C212000EFFF2F2AD8A08DD71200FFD7A8
:020000040030CA
:0300010006170ED1
:020005008580F4
:060008000FC00FE00F40E5
:00000001FF
